 getfldmdf004

 Timestamp is e7258cb2 (reproducible build file hash)

 Preferred load address is 0000000180000000

 Start         Length     Name                   Class
 0001:00000000 00002bd0H .text$mn                CODE
 0001:00002bd0 00000036H .text$mn$00             CODE
 0001:00002c06 00000092H .text$x                 CODE
 0002:00000000 00000198H .idata$5                DATA
 0002:00000198 00000038H .00cfg                  DATA
 0002:000001d0 00000008H .CRT$XCA                DATA
 0002:000001d8 00000008H .CRT$XCZ                DATA
 0002:000001e0 00000008H .CRT$XIA                DATA
 0002:000001e8 00000008H .CRT$XIC                DATA
 0002:000001f0 00000008H .CRT$XIZ                DATA
 0002:000001f8 00000008H .CRT$XLA                DATA
 0002:00000200 00000008H .CRT$XLZ                DATA
 0002:00000208 00000008H .CRT$XPA                DATA
 0002:00000210 00000008H .CRT$XPZ                DATA
 0002:00000218 00000008H .CRT$XTA                DATA
 0002:00000220 00000010H .CRT$XTZ                DATA
 0002:00000228 00000000H .gehcont$y              DATA
 0002:00000228 00000000H .gfids$y                DATA
 0002:00000230 00001cd0H .rdata                  DATA
 0002:00001f00 00000000H .rdata$CastGuardVftablesA DATA
 0002:00001f00 00000000H .rdata$CastGuardVftablesC DATA
 0002:00001f00 00000028H .rdata$T                DATA
 0002:00001f28 000000a4H .rdata$voltmd           DATA
 0002:00001fcc 0000031cH .rdata$zzzdbg           DATA
 0002:000022e8 00000008H .rtc$IAA                DATA
 0002:000022f0 00000008H .rtc$IZZ                DATA
 0002:000022f8 00000008H .rtc$TAA                DATA
 0002:00002300 00000008H .rtc$TZZ                DATA
 0002:00002308 00000004H .tls                    DATA
 0002:0000230c 00000004H .tls$                   DATA
 0002:00002310 00000008H .tls$ZZZ                DATA
 0002:00002318 000002e8H .xdata                  DATA
 0002:00002600 000003e4H .edata                  DATA
 0002:000029e4 00000064H .idata$2                DATA
 0002:00002a48 00000018H .idata$3                DATA
 0002:00002a60 00000198H .idata$4                DATA
 0002:00002bf8 0000041eH .idata$6                DATA
 0003:00000000 00000500H .data                   DATA
 0003:00000500 0001b238H .bss                    DATA
 0004:00000000 00000384H .pdata                  DATA

  Address         Publics by Value              Rva+Base               Lib:Object

 0000:00000000       __AbsoluteZero             0000000000000000     <absolute>
 0000:00000000       ___safe_se_handler_count   0000000000000000     <absolute>
 0000:00000000       ___safe_se_handler_table   0000000000000000     <absolute>
 0000:00000000       __arm64x_extra_rfe_table   0000000000000000     <absolute>
 0000:00000000       __arm64x_extra_rfe_table_size 0000000000000000     <absolute>
 0000:00000000       __arm64x_native_entrypoint 0000000000000000     <absolute>
 0000:00000000       __arm64x_redirection_metadata 0000000000000000     <absolute>
 0000:00000000       __arm64x_redirection_metadata_count 0000000000000000     <absolute>
 0000:00000000       __dynamic_value_reloc_table 0000000000000000     <absolute>
 0000:00000000       __enclave_config           0000000000000000     <absolute>
 0000:00000000       __guard_check_icall_a64n_fptr 0000000000000000     <absolute>
 0000:00000000       __guard_eh_cont_count      0000000000000000     <absolute>
 0000:00000000       __guard_eh_cont_table      0000000000000000     <absolute>
 0000:00000000       __guard_fids_count         0000000000000000     <absolute>
 0000:00000000       __guard_fids_table         0000000000000000     <absolute>
 0000:00000000       __guard_iat_count          0000000000000000     <absolute>
 0000:00000000       __guard_iat_table          0000000000000000     <absolute>
 0000:00000000       __guard_longjmp_count      0000000000000000     <absolute>
 0000:00000000       __guard_longjmp_table      0000000000000000     <absolute>
 0000:00000000       __hybrid_auxiliary_iat     0000000000000000     <absolute>
 0000:00000000       __hybrid_auxiliary_iat_copy 0000000000000000     <absolute>
 0000:00000000       __hybrid_code_map          0000000000000000     <absolute>
 0000:00000000       __hybrid_code_map_count    0000000000000000     <absolute>
 0000:00000000       __x64_code_ranges_to_entry_points 0000000000000000     <absolute>
 0000:00000000       __x64_code_ranges_to_entry_points_count 0000000000000000     <absolute>
 0000:00000100       __guard_flags              0000000000000100     <absolute>
 0000:00000000       __ImageBase                0000000180000000     <linker-defined>
 0001:00000000       ?NewObject@JNIEnv_@@QEAAPEAV_jobject@@PEAV_jclass@@PEAU_jmethodID@@ZZ 0000000180001000 f i libgetfldmdf004.obj
 0001:00000028       ?TranslateError@@YAPEBDW4jvmtiError@@@Z 0000000180001028 f   libgetfldmdf004.obj
 0001:000002e0       ?nsk_jni_check_exception@@YAHPEAUJNIEnv_@@QEBDH@Z 00000001800012e0 f   libgetfldmdf004.obj
 0001:00000424       ?nsk_jni_lverify@@YAHHPEAUJNIEnv_@@HQEBDH1ZZ 0000000180001424 f   libgetfldmdf004.obj
 0001:000004c4       Agent_Initialize           00000001800014c4 f   libgetfldmdf004.obj
 0001:00000538       Agent_OnAttach             0000000180001538 f   libgetfldmdf004.obj
 0001:00000538       Agent_OnLoad               0000000180001538 f   libgetfldmdf004.obj
 0001:00000540       Java_nsk_jvmti_GetFieldModifiers_getfldmdf004_check 0000000180001540 f   libgetfldmdf004.obj
 0001:00000688       Java_nsk_jvmti_GetFieldModifiers_getfldmdf004_getRes 0000000180001688 f   libgetfldmdf004.obj
 0001:00000690       Java_nsk_jvmti_unit_FollowReferences_FollowRefObjects_addRefToVerify 0000000180001690 f   libgetfldmdf004.obj
 0001:00000868       Java_nsk_jvmti_unit_FollowReferences_FollowRefObjects_getTag 0000000180001868 f   libgetfldmdf004.obj
 0001:00000928       Java_nsk_jvmti_unit_FollowReferences_FollowRefObjects_resetRefsToVerify 0000000180001928 f   libgetfldmdf004.obj
 0001:00000930       Java_nsk_jvmti_unit_FollowReferences_FollowRefObjects_resetTags 0000000180001930 f   libgetfldmdf004.obj
 0001:00000974       Java_nsk_jvmti_unit_FollowReferences_FollowRefObjects_setTag 0000000180001974 f   libgetfldmdf004.obj
 0001:00000bcc       Java_nsk_share_jvmti_ArgumentHandler_getAgentOptionsString 0000000180001bcc f   libgetfldmdf004.obj
 0001:00000c7c       Java_nsk_share_jvmti_DebugeeClass_checkStatus 0000000180001c7c f   libgetfldmdf004.obj
 0001:00000d04       Java_nsk_share_jvmti_DebugeeClass_resetAgentData 0000000180001d04 f   libgetfldmdf004.obj
 0001:00000d64       Java_nsk_share_jvmti_RedefineAgent_agentStatus 0000000180001d64 f   libgetfldmdf004.obj
 0001:00000d70       Java_nsk_share_jvmti_RedefineAgent_isRedefined 0000000180001d70 f   libgetfldmdf004.obj
 0001:00000d7c       Java_nsk_share_jvmti_RedefineAgent_redefineAttempted 0000000180001d7c f   libgetfldmdf004.obj
 0001:00000d88       MA_checkStatus             0000000180001d88 f   libgetfldmdf004.obj
 0001:00000e2c       __local_stdio_printf_options 0000000180001e2c f i libgetfldmdf004.obj
 0001:0000100c       exitOnError                000000018000200c f   libgetfldmdf004.obj
 0001:000010c0       fprintf                    00000001800020c0 f i libgetfldmdf004.obj
 0001:00001104       nsk_jvmti_lverify          0000000180002104 f   libgetfldmdf004.obj
 0001:000011f4       nsk_jvmti_resetAgentData   00000001800021f4 f   libgetfldmdf004.obj
 0001:00001274       nsk_jvmti_setFailStatus    0000000180002274 f   libgetfldmdf004.obj
 0001:000012b0       nsk_lcomplain              00000001800022b0 f   libgetfldmdf004.obj
 0001:000012d0       nsk_ldisplay               00000001800022d0 f   libgetfldmdf004.obj
 0001:000012f0       nsk_ltrace                 00000001800022f0 f   libgetfldmdf004.obj
 0001:00001310       nsk_lvcomplain             0000000180002310 f   libgetfldmdf004.obj
 0001:000014c8       nsk_lvdisplay              00000001800024c8 f   libgetfldmdf004.obj
 0001:00001514       nsk_lverify                0000000180002514 f   libgetfldmdf004.obj
 0001:00001570       nsk_lvtrace                0000000180002570 f   libgetfldmdf004.obj
 0001:000015d0       nsk_printf                 00000001800025d0 f   libgetfldmdf004.obj
 0001:000015f8       nsk_vprintf                00000001800025f8 f   libgetfldmdf004.obj
 0001:000016ac       printModifiers             00000001800026ac f   libgetfldmdf004.obj
 0001:00001784       printf                     0000000180002784 f i libgetfldmdf004.obj
 0001:00001cac       __raise_securityfailure    0000000180002cac f   MSVCRT:gs_report.obj
 0001:00001ce0       __report_gsfailure         0000000180002ce0 f   MSVCRT:gs_report.obj
 0001:00001f20       __GSHandlerCheck           0000000180002f20 f   MSVCRT:gshandler.obj
 0001:00001f40       __GSHandlerCheckCommon     0000000180002f40 f   MSVCRT:gshandler.obj
 0001:00001fb0       __security_check_cookie    0000000180002fb0 f   MSVCRT:amdsecgs.obj
 0001:000022f0       _DllMainCRTStartup         00000001800032f0 f   MSVCRT:dll_dllmain.obj
 0001:00002330       __scrt_acquire_startup_lock 0000000180003330 f   MSVCRT:utility.obj
 0001:0000236c       __scrt_dllmain_after_initialize_c 000000018000336c f   MSVCRT:utility.obj
 0001:000023a0       __scrt_dllmain_before_initialize_c 00000001800033a0 f   MSVCRT:utility.obj
 0001:000023b8       __scrt_dllmain_crt_thread_attach 00000001800033b8 f   MSVCRT:utility.obj
 0001:000023e0       __scrt_dllmain_crt_thread_detach 00000001800033e0 f   MSVCRT:utility.obj
 0001:000023f8       __scrt_dllmain_exception_filter 00000001800033f8 f   MSVCRT:utility.obj
 0001:00002458       __scrt_dllmain_uninitialize_c 0000000180003458 f   MSVCRT:utility.obj
 0001:00002488       __scrt_dllmain_uninitialize_critical 0000000180003488 f   MSVCRT:utility.obj
 0001:0000249c       __scrt_initialize_crt      000000018000349c f   MSVCRT:utility.obj
 0001:000024e8       __scrt_initialize_onexit_tables 00000001800034e8 f   MSVCRT:utility.obj
 0001:00002574       __scrt_is_nonwritable_in_current_image 0000000180003574 f   MSVCRT:utility.obj
 0001:0000260c       __scrt_release_startup_lock 000000018000360c f   MSVCRT:utility.obj
 0001:00002630       __scrt_uninitialize_crt    0000000180003630 f   MSVCRT:utility.obj
 0001:0000265c       _onexit                    000000018000365c f   MSVCRT:utility.obj
 0001:00002698       atexit                     0000000180003698 f   MSVCRT:utility.obj
 0001:000026b0       __crt_debugger_hook        00000001800036b0 f   MSVCRT:utility_desktop.obj
 0001:000026b8       __scrt_fastfail            00000001800036b8 f   MSVCRT:utility_desktop.obj
 0001:00002804       _guard_check_icall_nop     0000000180003804 f i MSVCRT:guard_support.obj
 0001:00002808       __security_init_cookie     0000000180003808 f   MSVCRT:gs_support.obj
 0001:000028b4       DllMain                    00000001800038b4 f   MSVCRT:dll_dllmain_stub.obj
 0001:000028d8       ?__scrt_initialize_type_info@@YAXXZ 00000001800038d8 f   MSVCRT:tncleanup.obj
 0001:000028e8       ?__scrt_uninitialize_type_info@@YAXXZ 00000001800038e8 f   MSVCRT:tncleanup.obj
 0001:000028f4       __local_stdio_scanf_options 00000001800038f4 f i MSVCRT:default_local_stdio_options.obj
 0001:000028fc       __scrt_initialize_default_local_stdio_options 00000001800038fc f   MSVCRT:default_local_stdio_options.obj
 0001:00002918       __scrt_get_dyn_tls_init_callback 0000000180003918 f   MSVCRT:dyn_tls_init.obj
 0001:00002920       _RTC_Initialize            0000000180003920 f   MSVCRT:initsect.obj
 0001:0000295c       _RTC_Terminate             000000018000395c f   MSVCRT:initsect.obj
 0001:00002998       __isa_available_init       0000000180003998 f   MSVCRT:cpu_disp.obj
 0001:00002b44       _get_startup_argv_mode     0000000180003b44 f   MSVCRT:argv_mode.obj
 0001:00002b4c       __scrt_is_ucrt_dll_in_use  0000000180003b4c f   MSVCRT:ucrt_detection.obj
 0001:00002b60       memcpy                     0000000180003b60 f   vcruntime:VCRUNTIME140.dll
 0001:00002b66       memset                     0000000180003b66 f   vcruntime:VCRUNTIME140.dll
 0001:00002b6c       strchr                     0000000180003b6c f   vcruntime:VCRUNTIME140.dll
 0001:00002b72       __C_specific_handler       0000000180003b72 f   vcruntime:VCRUNTIME140.dll
 0001:00002b78       __std_type_info_destroy_list 0000000180003b78 f   vcruntime:VCRUNTIME140.dll
 0001:00002b7e       strcmp                     0000000180003b7e f   ucrt:api-ms-win-crt-string-l1-1-0.dll
 0001:00002b84       strlen                     0000000180003b84 f   ucrt:api-ms-win-crt-string-l1-1-0.dll
 0001:00002b8a       _initterm                  0000000180003b8a f   ucrt:api-ms-win-crt-runtime-l1-1-0.dll
 0001:00002b90       _initterm_e                0000000180003b90 f   ucrt:api-ms-win-crt-runtime-l1-1-0.dll
 0001:00002b96       _seh_filter_dll            0000000180003b96 f   ucrt:api-ms-win-crt-runtime-l1-1-0.dll
 0001:00002b9c       _configure_narrow_argv     0000000180003b9c f   ucrt:api-ms-win-crt-runtime-l1-1-0.dll
 0001:00002ba2       _initialize_narrow_environment 0000000180003ba2 f   ucrt:api-ms-win-crt-runtime-l1-1-0.dll
 0001:00002ba8       _initialize_onexit_table   0000000180003ba8 f   ucrt:api-ms-win-crt-runtime-l1-1-0.dll
 0001:00002bae       _register_onexit_function  0000000180003bae f   ucrt:api-ms-win-crt-runtime-l1-1-0.dll
 0001:00002bb4       _execute_onexit_table      0000000180003bb4 f   ucrt:api-ms-win-crt-runtime-l1-1-0.dll
 0001:00002bba       _crt_atexit                0000000180003bba f   ucrt:api-ms-win-crt-runtime-l1-1-0.dll
 0001:00002bc0       _cexit                     0000000180003bc0 f   ucrt:api-ms-win-crt-runtime-l1-1-0.dll
 0001:00002bc8       __acrt_initialize          0000000180003bc8 f   MSVCRT:ucrt_stubs.obj
 0001:00002bc8       __acrt_thread_attach       0000000180003bc8 f   MSVCRT:ucrt_stubs.obj
 0001:00002bc8       __acrt_thread_detach       0000000180003bc8 f   MSVCRT:ucrt_stubs.obj
 0001:00002bc8       __acrt_uninitialize        0000000180003bc8 f   MSVCRT:ucrt_stubs.obj
 0001:00002bc8       __acrt_uninitialize_critical 0000000180003bc8 f   MSVCRT:ucrt_stubs.obj
 0001:00002bc8       __scrt_stub_for_acrt_initialize 0000000180003bc8 f   MSVCRT:ucrt_stubs.obj
 0001:00002bc8       __scrt_stub_for_acrt_thread_attach 0000000180003bc8 f   MSVCRT:ucrt_stubs.obj
 0001:00002bc8       __scrt_stub_for_acrt_thread_detach 0000000180003bc8 f   MSVCRT:ucrt_stubs.obj
 0001:00002bc8       __scrt_stub_for_acrt_uninitialize 0000000180003bc8 f   MSVCRT:ucrt_stubs.obj
 0001:00002bc8       __scrt_stub_for_acrt_uninitialize_critical 0000000180003bc8 f   MSVCRT:ucrt_stubs.obj
 0001:00002bc8       __vcrt_initialize          0000000180003bc8 f   MSVCRT:ucrt_stubs.obj
 0001:00002bc8       __vcrt_thread_attach       0000000180003bc8 f   MSVCRT:ucrt_stubs.obj
 0001:00002bc8       __vcrt_thread_detach       0000000180003bc8 f   MSVCRT:ucrt_stubs.obj
 0001:00002bc8       __vcrt_uninitialize        0000000180003bc8 f   MSVCRT:ucrt_stubs.obj
 0001:00002bc8       __vcrt_uninitialize_critical 0000000180003bc8 f   MSVCRT:ucrt_stubs.obj
 0001:00002bcc       __scrt_stub_for_is_c_termination_complete 0000000180003bcc f   MSVCRT:ucrt_stubs.obj
 0001:00002bcc       _is_c_termination_complete 0000000180003bcc f   MSVCRT:ucrt_stubs.obj
 0001:00002be0       _guard_dispatch_icall_nop  0000000180003be0 f   MSVCRT:guard_dispatch.obj
 0001:00002c00       _guard_xfg_dispatch_icall_nop 0000000180003c00 f   MSVCRT:guard_xfg_dispatch.obj
 0002:00000000       __imp_RtlCaptureContext    0000000180004000     kernel32:KERNEL32.dll
 0002:00000008       __imp_RtlLookupFunctionEntry 0000000180004008     kernel32:KERNEL32.dll
 0002:00000010       __imp_RtlVirtualUnwind     0000000180004010     kernel32:KERNEL32.dll
 0002:00000018       __imp_UnhandledExceptionFilter 0000000180004018     kernel32:KERNEL32.dll
 0002:00000020       __imp_SetUnhandledExceptionFilter 0000000180004020     kernel32:KERNEL32.dll
 0002:00000028       __imp_GetCurrentProcess    0000000180004028     kernel32:KERNEL32.dll
 0002:00000030       __imp_TerminateProcess     0000000180004030     kernel32:KERNEL32.dll
 0002:00000038       __imp_IsProcessorFeaturePresent 0000000180004038     kernel32:KERNEL32.dll
 0002:00000040       __imp_CloseHandle          0000000180004040     kernel32:KERNEL32.dll
 0002:00000048       __imp_InitializeCriticalSectionAndSpinCount 0000000180004048     kernel32:KERNEL32.dll
 0002:00000050       __imp_DeleteCriticalSection 0000000180004050     kernel32:KERNEL32.dll
 0002:00000058       __imp_CreateEventW         0000000180004058     kernel32:KERNEL32.dll
 0002:00000060       __imp_GetModuleHandleW     0000000180004060     kernel32:KERNEL32.dll
 0002:00000068       __imp_GetProcAddress       0000000180004068     kernel32:KERNEL32.dll
 0002:00000070       __imp_IsDebuggerPresent    0000000180004070     kernel32:KERNEL32.dll
 0002:00000078       __imp_QueryPerformanceCounter 0000000180004078     kernel32:KERNEL32.dll
 0002:00000080       __imp_GetCurrentProcessId  0000000180004080     kernel32:KERNEL32.dll
 0002:00000088       __imp_GetCurrentThreadId   0000000180004088     kernel32:KERNEL32.dll
 0002:00000090       __imp_GetSystemTimeAsFileTime 0000000180004090     kernel32:KERNEL32.dll
 0002:00000098       __imp_DisableThreadLibraryCalls 0000000180004098     kernel32:KERNEL32.dll
 0002:000000a0       __imp_InitializeSListHead  00000001800040a0     kernel32:KERNEL32.dll
 0002:000000a8       \177KERNEL32_NULL_THUNK_DATA 00000001800040a8     kernel32:KERNEL32.dll
 0002:000000b0       __imp_memcpy               00000001800040b0     vcruntime:VCRUNTIME140.dll
 0002:000000b8       __imp_memset               00000001800040b8     vcruntime:VCRUNTIME140.dll
 0002:000000c0       __imp_strchr               00000001800040c0     vcruntime:VCRUNTIME140.dll
 0002:000000c8       __imp___C_specific_handler 00000001800040c8     vcruntime:VCRUNTIME140.dll
 0002:000000d0       __imp___std_type_info_destroy_list 00000001800040d0     vcruntime:VCRUNTIME140.dll
 0002:000000d8       \177VCRUNTIME140_NULL_THUNK_DATA 00000001800040d8     vcruntime:VCRUNTIME140.dll
 0002:000000e0       __imp__errno               00000001800040e0     ucrt:api-ms-win-crt-runtime-l1-1-0.dll
 0002:000000e8       __imp_exit                 00000001800040e8     ucrt:api-ms-win-crt-runtime-l1-1-0.dll
 0002:000000f0       __imp__cexit               00000001800040f0     ucrt:api-ms-win-crt-runtime-l1-1-0.dll
 0002:000000f8       __imp__crt_atexit          00000001800040f8     ucrt:api-ms-win-crt-runtime-l1-1-0.dll
 0002:00000100       __imp__execute_onexit_table 0000000180004100     ucrt:api-ms-win-crt-runtime-l1-1-0.dll
 0002:00000108       __imp__register_onexit_function 0000000180004108     ucrt:api-ms-win-crt-runtime-l1-1-0.dll
 0002:00000110       __imp__initialize_onexit_table 0000000180004110     ucrt:api-ms-win-crt-runtime-l1-1-0.dll
 0002:00000118       __imp__initialize_narrow_environment 0000000180004118     ucrt:api-ms-win-crt-runtime-l1-1-0.dll
 0002:00000120       __imp__configure_narrow_argv 0000000180004120     ucrt:api-ms-win-crt-runtime-l1-1-0.dll
 0002:00000128       __imp__seh_filter_dll      0000000180004128     ucrt:api-ms-win-crt-runtime-l1-1-0.dll
 0002:00000130       __imp__initterm_e          0000000180004130     ucrt:api-ms-win-crt-runtime-l1-1-0.dll
 0002:00000138       __imp__initterm            0000000180004138     ucrt:api-ms-win-crt-runtime-l1-1-0.dll
 0002:00000140       \177api-ms-win-crt-runtime-l1-1-0_NULL_THUNK_DATA 0000000180004140     ucrt:api-ms-win-crt-runtime-l1-1-0.dll
 0002:00000148       __imp___acrt_iob_func      0000000180004148     ucrt:api-ms-win-crt-stdio-l1-1-0.dll
 0002:00000150       __imp_fflush               0000000180004150     ucrt:api-ms-win-crt-stdio-l1-1-0.dll
 0002:00000158       __imp___stdio_common_vsprintf 0000000180004158     ucrt:api-ms-win-crt-stdio-l1-1-0.dll
 0002:00000160       __imp___stdio_common_vfprintf 0000000180004160     ucrt:api-ms-win-crt-stdio-l1-1-0.dll
 0002:00000168       \177api-ms-win-crt-stdio-l1-1-0_NULL_THUNK_DATA 0000000180004168     ucrt:api-ms-win-crt-stdio-l1-1-0.dll
 0002:00000170       __imp_strcmp               0000000180004170     ucrt:api-ms-win-crt-string-l1-1-0.dll
 0002:00000178       __imp__strdup              0000000180004178     ucrt:api-ms-win-crt-string-l1-1-0.dll
 0002:00000178       __imp_strdup               0000000180004178     ucrt:api-ms-win-crt-string-l1-1-0.dll
 0002:00000180       __imp_strlen               0000000180004180     ucrt:api-ms-win-crt-string-l1-1-0.dll
 0002:00000188       __imp_strncpy              0000000180004188     ucrt:api-ms-win-crt-string-l1-1-0.dll
 0002:00000190       \177api-ms-win-crt-string-l1-1-0_NULL_THUNK_DATA 0000000180004190     ucrt:api-ms-win-crt-string-l1-1-0.dll
 0002:00000198       __guard_check_icall_fptr   0000000180004198     MSVCRT:guard_support.obj
 0002:000001a0       __guard_xfg_check_icall_fptr 00000001800041a0     MSVCRT:guard_support.obj
 0002:000001a8       __guard_dispatch_icall_fptr 00000001800041a8     MSVCRT:guard_support.obj
 0002:000001b0       __guard_xfg_dispatch_icall_fptr 00000001800041b0     MSVCRT:guard_support.obj
 0002:000001b8       __guard_xfg_table_dispatch_icall_fptr 00000001800041b8     MSVCRT:guard_support.obj
 0002:000001c0       __castguard_check_failure_os_handled_fptr 00000001800041c0     MSVCRT:guard_support.obj
 0002:000001c8       __guard_memcpy_fptr        00000001800041c8     vcruntime:softmemtag.obj
 0002:000001d0       __xc_a                     00000001800041d0     MSVCRT:initializers.obj
 0002:000001d8       __xc_z                     00000001800041d8     MSVCRT:initializers.obj
 0002:000001e0       __xi_a                     00000001800041e0     MSVCRT:initializers.obj
 0002:000001f0       __xi_z                     00000001800041f0     MSVCRT:initializers.obj
 0002:000001f8       __xl_a                     00000001800041f8     MSVCRT:tlssup.obj
 0002:00000200       __xl_z                     0000000180004200     MSVCRT:tlssup.obj
 0002:00000208       __xp_a                     0000000180004208     MSVCRT:initializers.obj
 0002:00000210       __xp_z                     0000000180004210     MSVCRT:initializers.obj
 0002:00000218       __xt_a                     0000000180004218     MSVCRT:initializers.obj
 0002:00000220       __xt_z                     0000000180004220     MSVCRT:initializers.obj
 0002:00000230       g_refKindStr               0000000180004230     libgetfldmdf004.obj
 0002:000003e0       ??_C@_09BPLDFGCI@unknown_0@ 00000001800043e0     libgetfldmdf004.obj
 0002:000003f0       ??_C@_0BL@FPNMECJD@JVMTI_HEAP_REFERENCE_CLASS@ 00000001800043f0     libgetfldmdf004.obj
 0002:00000410       ??_C@_0BL@FKGKKLNM@JVMTI_HEAP_REFERENCE_FIELD@ 0000000180004410     libgetfldmdf004.obj
 0002:00000430       ??_C@_0CD@CAEHCFJF@JVMTI_HEAP_REFERENCE_ARRAY_ELEM@ 0000000180004430     libgetfldmdf004.obj
 0002:00000458       ??_C@_0CC@DNEBMCNK@JVMTI_HEAP_REFERENCE_CLASS_LOAD@ 0000000180004458     libgetfldmdf004.obj
 0002:00000480       ??_C@_0BN@CJMIPEBB@JVMTI_HEAP_REFERENCE_SIGNERS@ 0000000180004480     libgetfldmdf004.obj
 0002:000004a0       ??_C@_0CH@HBOIDPEB@JVMTI_HEAP_REFERENCE_PROTECTION@ 00000001800044a0     libgetfldmdf004.obj
 0002:000004c8       ??_C@_0BP@MDKGDGKL@JVMTI_HEAP_REFERENCE_INTERFACE@ 00000001800044c8     libgetfldmdf004.obj
 0002:000004e8       ??_C@_0CC@JJMIHNJH@JVMTI_HEAP_REFERENCE_STATIC_FIE@ 00000001800044e8     libgetfldmdf004.obj
 0002:00000510       ??_C@_0CD@IDHEEGID@JVMTI_HEAP_REFERENCE_CONSTANT_P@ 0000000180004510     libgetfldmdf004.obj
 0002:00000538       ??_C@_0CA@EFFCHNG@JVMTI_HEAP_REFERENCE_SUPERCLASS@ 0000000180004538     libgetfldmdf004.obj
 0002:00000558       ??_C@_0L@PCDFHGCJ@unknown_11@ 0000000180004558     libgetfldmdf004.obj
 0002:00000568       ??_C@_0L@NJBICFOK@unknown_12@ 0000000180004568     libgetfldmdf004.obj
 0002:00000578       ??_C@_0L@MAADBEKL@unknown_13@ 0000000180004578     libgetfldmdf004.obj
 0002:00000588       ??_C@_0L@IPECICGM@unknown_14@ 0000000180004588     libgetfldmdf004.obj
 0002:00000598       ??_C@_0L@JGFJLDCN@unknown_15@ 0000000180004598     libgetfldmdf004.obj
 0002:000005a8       ??_C@_0L@LNHEOAOO@unknown_16@ 00000001800045a8     libgetfldmdf004.obj
 0002:000005b8       ??_C@_0L@KEGPNBKP@unknown_17@ 00000001800045b8     libgetfldmdf004.obj
 0002:000005c8       ??_C@_0L@CDPHMNGA@unknown_18@ 00000001800045c8     libgetfldmdf004.obj
 0002:000005d8       ??_C@_0L@DKOMPMCB@unknown_19@ 00000001800045d8     libgetfldmdf004.obj
 0002:000005e8       ??_C@_0L@OJGIPJDB@unknown_20@ 00000001800045e8     libgetfldmdf004.obj
 0002:000005f8       ??_C@_0CA@KAOFNDEM@JVMTI_HEAP_REFERENCE_JNI_GLOBAL@ 00000001800045f8     libgetfldmdf004.obj
 0002:00000618       ??_C@_0CC@HPFAJBK@JVMTI_HEAP_REFERENCE_SYSTEM_CLA@ 0000000180004618     libgetfldmdf004.obj
 0002:00000640       ??_C@_0BN@FDEGFOHC@JVMTI_HEAP_REFERENCE_MONITOR@ 0000000180004640     libgetfldmdf004.obj
 0002:00000660       ??_C@_0CB@HKIBCMAJ@JVMTI_HEAP_REFERENCE_STACK_LOCA@ 0000000180004660     libgetfldmdf004.obj
 0002:00000688       ??_C@_0BP@EAACMMOE@JVMTI_HEAP_REFERENCE_JNI_LOCAL@ 0000000180004688     libgetfldmdf004.obj
 0002:000006a8       ??_C@_0BM@IJDEOGOE@JVMTI_HEAP_REFERENCE_THREAD@ 00000001800046a8     libgetfldmdf004.obj
 0002:000006c8       ??_C@_0BL@EDGPPKC@JVMTI_HEAP_REFERENCE_OTHER@ 00000001800046c8     libgetfldmdf004.obj
 0002:000006e4       ??_C@_04BCJPDBDA@Code@     00000001800046e4     libgetfldmdf004.obj
 0002:000006f0       ??_C@_0BA@OCLMCFKC@LineNumberTable@ 00000001800046f0     libgetfldmdf004.obj
 0002:00000700       ??_C@_0BD@CPAEPILC@LocalVariableTable@ 0000000180004700     libgetfldmdf004.obj
 0002:00000718       ??_C@_0BH@NMBDNHBD@LocalVariableTypeTable@ 0000000180004718     libgetfldmdf004.obj
 0002:00000730       ??_C@_0O@HIHEEDNJ@StackMapTable@ 0000000180004730     libgetfldmdf004.obj
 0002:00000740       ??_C@_06BFLEOCEF@field0@   0000000180004740     libgetfldmdf004.obj
 0002:00000748       ??_C@_01JPJNBJEM@I@        0000000180004748     libgetfldmdf004.obj
 0002:0000074c       ??_C@_06MKPNDAE@field1@    000000018000474c     libgetfldmdf004.obj
 0002:00000754       ??_C@_06CHICIAMH@field2@   0000000180004754     libgetfldmdf004.obj
 0002:0000075c       ??_C@_06DOJJLBIG@field3@   000000018000475c     libgetfldmdf004.obj
 0002:00000764       ??_C@_06HBNICHEB@field4@   0000000180004764     libgetfldmdf004.obj
 0002:0000076c       ??_C@_06GIMDBGAA@field5@   000000018000476c     libgetfldmdf004.obj
 0002:00000774       ??_C@_06EDOOEFMD@field6@   0000000180004774     libgetfldmdf004.obj
 0002:0000077c       ??_C@_06FKPFHEIC@field7@   000000018000477c     libgetfldmdf004.obj
 0002:00000784       ??_C@_06NNGNGIEN@field8@   0000000180004784     libgetfldmdf004.obj
 0002:0000078c       ??_C@_06MEHGFJAM@field9@   000000018000478c     libgetfldmdf004.obj
 0002:00000798       ??_C@_07NICHFNDJ@field10@  0000000180004798     libgetfldmdf004.obj
 0002:000007a0       ??_C@_07MBDMGMHI@field11@  00000001800047a0     libgetfldmdf004.obj
 0002:000007a8       ??_C@_07OKBBDPLL@field12@  00000001800047a8     libgetfldmdf004.obj
 0002:000007b0       ??_C@_07PDAKAOPK@field13@  00000001800047b0     libgetfldmdf004.obj
 0002:000007b8       ??_C@_07LMELJIDN@field14@  00000001800047b8     libgetfldmdf004.obj
 0002:000007c0       ??_C@_07KFFAKJHM@field15@  00000001800047c0     libgetfldmdf004.obj
 0002:000007c8       ??_C@_07IOHNPKLP@field16@  00000001800047c8     libgetfldmdf004.obj
 0002:000007d0       ??_C@_07JHGGMLPO@field17@  00000001800047d0     libgetfldmdf004.obj
 0002:000007d8       ??_C@_07BAPONHDB@field18@  00000001800047d8     libgetfldmdf004.obj
 0002:000007e0       ??_C@_07JOFOGHA@field19@   00000001800047e0     libgetfldmdf004.obj
 0002:000007e8       ??_C@_07NKGBODGA@field20@  00000001800047e8     libgetfldmdf004.obj
 0002:000007f0       ??_C@_07MDHKNCCB@field21@  00000001800047f0     libgetfldmdf004.obj
 0002:000007f8       ??_C@_07OIFHIBOC@field22@  00000001800047f8     libgetfldmdf004.obj
 0002:00000800       ??_C@_07PBEMLAKD@field23@  0000000180004800     libgetfldmdf004.obj
 0002:00000808       ??_C@_07LOANCGGE@field24@  0000000180004808     libgetfldmdf004.obj
 0002:00000810       ??_C@_07KHBGBHCF@field25@  0000000180004810     libgetfldmdf004.obj
 0002:00000818       ??_C@_07IMDLEEOG@field26@  0000000180004818     libgetfldmdf004.obj
 0002:00000820       ??_C@_07JFCAHFKH@field27@  0000000180004820     libgetfldmdf004.obj
 0002:00000828       ??_C@_07BCLIGJGI@field28@  0000000180004828     libgetfldmdf004.obj
 0002:00000830       ??_C@_07LKDFICJ@field29@   0000000180004830     libgetfldmdf004.obj
 0002:00000838       ??_C@_07NLKDIJFH@field30@  0000000180004838     libgetfldmdf004.obj
 0002:00000840       ??_C@_07MCLILIBG@field31@  0000000180004840     libgetfldmdf004.obj
 0002:00000848       ??_C@_07OJJFOLNF@field32@  0000000180004848     libgetfldmdf004.obj
 0002:00000850       ??_C@_07PAIONKJE@field33@  0000000180004850     libgetfldmdf004.obj
 0002:00000858       ??_C@_07LPMPEMFD@field34@  0000000180004858     libgetfldmdf004.obj
 0002:00000860       ??_C@_07KGNEHNBC@field35@  0000000180004860     libgetfldmdf004.obj
 0002:00000868       ??_C@_07INPJCONB@field36@  0000000180004868     libgetfldmdf004.obj
 0002:00000870       ??_C@_07JEOCBPJA@field37@  0000000180004870     libgetfldmdf004.obj
 0002:00000878       ??_C@_07BDHKADFP@field38@  0000000180004878     libgetfldmdf004.obj
 0002:00000880       ??_C@_07KGBDCBO@field39@   0000000180004880     libgetfldmdf004.obj
 0002:00000888       ??_C@_07NOOMJPNC@field40@  0000000180004888     libgetfldmdf004.obj
 0002:00000890       ??_C@_07MHPHKOJD@field41@  0000000180004890     libgetfldmdf004.obj
 0002:00000898       ??_C@_07OMNKPNFA@field42@  0000000180004898     libgetfldmdf004.obj
 0002:000008a0       ??_C@_07PFMBMMBB@field43@  00000001800048a0     libgetfldmdf004.obj
 0002:000008a8       ??_C@_07LKIAFKNG@field44@  00000001800048a8     libgetfldmdf004.obj
 0002:000008b0       ??_C@_07KDJLGLJH@field45@  00000001800048b0     libgetfldmdf004.obj
 0002:000008b8       ??_C@_07IILGDIFE@field46@  00000001800048b8     libgetfldmdf004.obj
 0002:000008c0       ??_C@_07JBKNAJBF@field47@  00000001800048c0     libgetfldmdf004.obj
 0002:000008c8       ??_C@_0L@HCDIAMJG@?9?5?$CFs?0?5?$CFd?3?5@ 00000001800048c8     libgetfldmdf004.obj
 0002:000008e0       ??_C@_0JI@HLPECLFI@?$CD?5?4?4?4?6?$CD?5ERROR?3?5too?5many?5complai@ 00000001800048e0     libgetfldmdf004.obj
 0002:00000980       ??_C@_0ED@JNEKCCOB@The?5following?5fake?5exception?5st@ 0000000180004980     libgetfldmdf004.obj
 0002:000009c8       ??_C@_0CN@FCNMDFBH@nsk?4share?4Fake_Exception_for_RU@ 00000001800049c8     libgetfldmdf004.obj
 0002:000009f8       ??_C@_08PGFFNAEI@?$CI?$CFs?3?$CFd?$CJ?5@ 00000001800049f8     libgetfldmdf004.obj
 0002:00000a08       ??_C@_0DP@IENMAEGI@s?2test?2hotspot?2jtreg?2vmTestbase@ 0000000180004a08     libgetfldmdf004.obj
 0002:00000a48       ??_C@_0BL@NDJLFFJB@?7at?5nsk_lvcomplain?$CI?$CFs?3?$CFd?$CJ?6@ 0000000180004a48     libgetfldmdf004.obj
 0002:00000a68       ??_C@_0BC@JOOKAFKF@?$CD?5ERROR?3?5?$CFs?0?5?$CFd?3?5@ 0000000180004a68     libgetfldmdf004.obj
 0002:00000a80       ??_C@_09KJEAHMEH@?$CD?5ERROR?3?5@ 0000000180004a80     libgetfldmdf004.obj
 0002:00000a8c       ??_C@_02GPIOPFAK@?$DO?$DO@ 0000000180004a8c     libgetfldmdf004.obj
 0002:00000a90       ??_C@_02FODMEDOG@?$DM?$DM@ 0000000180004a90     libgetfldmdf004.obj
 0002:00000a94       ??_C@_02DJGKEECL@?4?4@     0000000180004a94     libgetfldmdf004.obj
 0002:00000a98       ??_C@_0O@CJPGJOAF@?9?5?$CFs?0?5?$CFd?3?5?$CFs?5@ 0000000180004a98     libgetfldmdf004.obj
 0002:00000aa8       ??_C@_0CB@IAKPDOIC@?$CD?5?5?5verified?5assertion?5is?5FALSE@ 0000000180004aa8     libgetfldmdf004.obj
 0002:00000ad0       ??_C@_0CO@LGONDEPD@stdout?3?5fflush?5failed?5?9?5err?$DN?$CFd?5@ 0000000180004ad0     libgetfldmdf004.obj
 0002:00000b00       ??_C@_0CO@KBGKJPBD@stderr?3?5fflush?5failed?5?9?5err?$DN?$CFd?5@ 0000000180004b00     libgetfldmdf004.obj
 0002:00000b30       ??_C@_0BB@JCNMKLLK@JVMTI_ERROR_NONE@ 0000000180004b30     libgetfldmdf004.obj
 0002:00000b48       ??_C@_0BL@LDIMKLPH@JVMTI_ERROR_INVALID_THREAD@ 0000000180004b48     libgetfldmdf004.obj
 0002:00000b68       ??_C@_0CB@PJFPAIKJ@JVMTI_ERROR_INVALID_THREAD_GROU@ 0000000180004b68     libgetfldmdf004.obj
 0002:00000b90       ??_C@_0BN@LLMKHMNF@JVMTI_ERROR_INVALID_PRIORITY@ 0000000180004b90     libgetfldmdf004.obj
 0002:00000bb0       ??_C@_0CB@MBOFKAGB@JVMTI_ERROR_THREAD_NOT_SUSPENDE@ 0000000180004bb0     libgetfldmdf004.obj
 0002:00000bd8       ??_C@_0BN@FABOLPBI@JVMTI_ERROR_THREAD_SUSPENDED@ 0000000180004bd8     libgetfldmdf004.obj
 0002:00000bf8       ??_C@_0BN@FDGNOBJM@JVMTI_ERROR_THREAD_NOT_ALIVE@ 0000000180004bf8     libgetfldmdf004.obj
 0002:00000c18       ??_C@_0BL@GOBIFKNJ@JVMTI_ERROR_INVALID_OBJECT@ 0000000180004c18     libgetfldmdf004.obj
 0002:00000c38       ??_C@_0BK@FCMAJPPC@JVMTI_ERROR_INVALID_CLASS@ 0000000180004c38     libgetfldmdf004.obj
 0002:00000c58       ??_C@_0BP@IKLLBKEB@JVMTI_ERROR_CLASS_NOT_PREPARED@ 0000000180004c58     libgetfldmdf004.obj
 0002:00000c78       ??_C@_0BN@KLPPLKG@JVMTI_ERROR_INVALID_METHODID@ 0000000180004c78     libgetfldmdf004.obj
 0002:00000c98       ??_C@_0BN@BCEKOKND@JVMTI_ERROR_INVALID_LOCATION@ 0000000180004c98     libgetfldmdf004.obj
 0002:00000cb8       ??_C@_0BM@DFDGPME@JVMTI_ERROR_INVALID_FIELDID@ 0000000180004cb8     libgetfldmdf004.obj
 0002:00000cd8       ??_C@_0BL@NELIEPEC@JVMTI_ERROR_NO_MORE_FRAMES@ 0000000180004cd8     libgetfldmdf004.obj
 0002:00000cf8       ??_C@_0BJ@BDBECFDM@JVMTI_ERROR_OPAQUE_FRAME@ 0000000180004cf8     libgetfldmdf004.obj
 0002:00000d18       ??_C@_0BK@MIIFNLOB@JVMTI_ERROR_TYPE_MISMATCH@ 0000000180004d18     libgetfldmdf004.obj
 0002:00000d38       ??_C@_0BJ@HPCAOILC@JVMTI_ERROR_INVALID_SLOT@ 0000000180004d38     libgetfldmdf004.obj
 0002:00000d58       ??_C@_0BG@CHILOPNI@JVMTI_ERROR_DUPLICATE@ 0000000180004d58     libgetfldmdf004.obj
 0002:00000d70       ??_C@_0BG@DIEMLHKM@JVMTI_ERROR_NOT_FOUND@ 0000000180004d70     libgetfldmdf004.obj
 0002:00000d88       ??_C@_0BM@NHMCKHOB@JVMTI_ERROR_INVALID_MONITOR@ 0000000180004d88     libgetfldmdf004.obj
 0002:00000da8       ??_C@_0BO@PPEDAJGL@JVMTI_ERROR_NOT_MONITOR_OWNER@ 0000000180004da8     libgetfldmdf004.obj
 0002:00000dc8       ??_C@_0BG@FCAIPEID@JVMTI_ERROR_INTERRUPT@ 0000000180004dc8     libgetfldmdf004.obj
 0002:00000de0       ??_C@_0CB@EGDBNKOI@JVMTI_ERROR_INVALID_CLASS_FORMA@ 0000000180004de0     libgetfldmdf004.obj
 0002:00000e08       ??_C@_0CG@DGKOGIAL@JVMTI_ERROR_CIRCULAR_CLASS_DEFI@ 0000000180004e08     libgetfldmdf004.obj
 0002:00000e30       ??_C@_0BP@ICEALPKC@JVMTI_ERROR_FAILS_VERIFICATION@ 0000000180004e30     libgetfldmdf004.obj
 0002:00000e50       ??_C@_0DC@JDACLMIO@JVMTI_ERROR_UNSUPPORTED_REDEFIN@ 0000000180004e50     libgetfldmdf004.obj
 0002:00000e88       ??_C@_0DE@GKDKNOMJ@JVMTI_ERROR_UNSUPPORTED_REDEFIN@ 0000000180004e88     libgetfldmdf004.obj
 0002:00000ec0       ??_C@_0BO@LAFKIOG@JVMTI_ERROR_INVALID_TYPESTATE@ 0000000180004ec0     libgetfldmdf004.obj
 0002:00000ee0       ??_C@_0DH@INDGCLLB@JVMTI_ERROR_UNSUPPORTED_REDEFIN@ 0000000180004ee0     libgetfldmdf004.obj
 0002:00000f18       ??_C@_0DE@NHEOMMGI@JVMTI_ERROR_UNSUPPORTED_REDEFIN@ 0000000180004f18     libgetfldmdf004.obj
 0002:00000f50       ??_C@_0CA@EKPNJOEP@JVMTI_ERROR_UNSUPPORTED_VERSION@ 0000000180004f50     libgetfldmdf004.obj
 0002:00000f70       ??_C@_0BN@OFFMAHHL@JVMTI_ERROR_NAMES_DONT_MATCH@ 0000000180004f70     libgetfldmdf004.obj
 0002:00000f90       ??_C@_0DN@HHBBLAKE@JVMTI_ERROR_UNSUPPORTED_REDEFIN@ 0000000180004f90     libgetfldmdf004.obj
 0002:00000fd0       ??_C@_0DO@HMBGBGNA@JVMTI_ERROR_UNSUPPORTED_REDEFIN@ 0000000180004fd0     libgetfldmdf004.obj
 0002:00001010       ??_C@_0BP@PBECGKHJ@JVMTI_ERROR_UNMODIFIABLE_CLASS@ 0000000180005010     libgetfldmdf004.obj
 0002:00001030       ??_C@_0BK@CANILEHF@JVMTI_ERROR_NOT_AVAILABLE@ 0000000180005030     libgetfldmdf004.obj
 0002:00001050       ??_C@_0CE@INJKMEFK@JVMTI_ERROR_MUST_POSSESS_CAPABI@ 0000000180005050     libgetfldmdf004.obj
 0002:00001078       ??_C@_0BJ@LBFPFPDM@JVMTI_ERROR_NULL_POINTER@ 0000000180005078     libgetfldmdf004.obj
 0002:00001098       ??_C@_0BP@CHJPNNEM@JVMTI_ERROR_ABSENT_INFORMATION@ 0000000180005098     libgetfldmdf004.obj
 0002:000010b8       ??_C@_0BP@OMFMNLC@JVMTI_ERROR_INVALID_EVENT_TYPE@ 00000001800050b8     libgetfldmdf004.obj
 0002:000010d8       ??_C@_0BN@BIBNPHHO@JVMTI_ERROR_ILLEGAL_ARGUMENT@ 00000001800050d8     libgetfldmdf004.obj
 0002:000010f8       ??_C@_0BK@KKNDHDCE@JVMTI_ERROR_NATIVE_METHOD@ 00000001800050f8     libgetfldmdf004.obj
 0002:00001118       ??_C@_0BK@PMKCFHAE@JVMTI_ERROR_OUT_OF_MEMORY@ 0000000180005118     libgetfldmdf004.obj
 0002:00001138       ??_C@_0BK@NNJBDMNB@JVMTI_ERROR_ACCESS_DENIED@ 0000000180005138     libgetfldmdf004.obj
 0002:00001158       ??_C@_0BI@GHECLMNC@JVMTI_ERROR_WRONG_PHASE@ 0000000180005158     libgetfldmdf004.obj
 0002:00001170       ??_C@_0BF@OLIHJOII@JVMTI_ERROR_INTERNAL@ 0000000180005170     libgetfldmdf004.obj
 0002:00001188       ??_C@_0BO@EOHGKJHI@JVMTI_ERROR_UNATTACHED_THREAD@ 0000000180005188     libgetfldmdf004.obj
 0002:000011a8       ??_C@_0CA@LKHFDACL@JVMTI_ERROR_INVALID_ENVIRONMENT@ 00000001800051a8     libgetfldmdf004.obj
 0002:000011c8       ??_C@_0BA@MMFHLOKK@?$DMunknown?5error?$DO@ 00000001800051c8     libgetfldmdf004.obj
 0002:000011d8       ??_C@_0CF@CBHOKDB@throwable?5?$DN?5jni?9?$DOExceptionOccur@ 00000001800051d8     libgetfldmdf004.obj
 0002:00001200       ??_C@_03OFAPEBGM@?$CFs?6@  0000000180005200     libgetfldmdf004.obj
 0002:00001208       ??_C@_0DM@LPIGEGNJ@s?2test?2hotspot?2jtreg?2vmTestbase@ 0000000180005208     libgetfldmdf004.obj
 0002:00001248       ??_C@_0CC@NFCNPEPK@Exception?5in?5JNI?5call?5?$CIcleared?$CJ@ 0000000180005248     libgetfldmdf004.obj
 0002:00001270       ??_C@_0BJ@IBAKFIKF@jni?9?$DOExceptionDescribe?$CI?$CJ@ 0000000180005270     libgetfldmdf004.obj
 0002:00001290       ??_C@_0BG@GGKALKMH@jni?9?$DOExceptionClear?$CI?$CJ@ 0000000180005290     libgetfldmdf004.obj
 0002:000012a8       ??_C@_0CF@JMGFGJLJ@?$CD?5?5?5verified?5JNI?5assertion?5is?5F@ 00000001800052a8     libgetfldmdf004.obj
 0002:000012d0       ??_C@_0CB@MLNJNCLJ@?5?5jvmti?5error?3?5code?$DN?$CFd?0?5name?$DN?$CFs@ 00000001800052d0     libgetfldmdf004.obj
 0002:000012f8       ??_C@_0CD@OHBGDKMK@?$CD?5?5?5jvmti?5error?3?5code?$DN?$CFd?0?5name?$DN@ 00000001800052f8     libgetfldmdf004.obj
 0002:00001320       ??_C@_0CG@JNNCGPHB@?$CD?5?5?5error?5expected?3?5code?$DN?$CFd?0?5na@ 0000000180005320     libgetfldmdf004.obj
 0002:00001350       ??_C@_0EB@IMGKPCGE@?$CIstr_obj?5?$DN?5jni?9?$DONewStringUTF?$CIco@ 0000000180005350     libgetfldmdf004.obj
 0002:000013a0       ??_C@_0EA@HFOGGBCC@s?2test?2hotspot?2jtreg?2vmTestbase@ 00000001800053a0     libgetfldmdf004.obj
 0002:000013e0       ??_C@_05KKCIMGE@error@     00000001800053e0     libgetfldmdf004.obj
 0002:000013e8       ??_C@_0CJ@JACLEAA@Test?5failed?5by?5setFailStatus?$CI?$CJ?4@ 00000001800053e8     libgetfldmdf004.obj
 0002:00001420       ??_C@_0EA@PNBCDMOA@s?2test?2hotspot?2jtreg?2vmTestbase@ 0000000180005420     libgetfldmdf004.obj
 0002:00001460       ??_C@_0DI@ILAHDLMP@?$CI?$CKagentThreadProc?$CJ?$CIjvmti_env?0?5a@ 0000000180005460     libgetfldmdf004.obj
 0002:00001498       ??_C@_0BD@KDBALNLB@JVMTI?5agent?5thread@ 0000000180005498     libgetfldmdf004.obj
 0002:000014b0       ??_C@_0BB@NOKBFPFO@java?1lang?1Thread@ 00000001800054b0     libgetfldmdf004.obj
 0002:000014c4       ??_C@_06FALKBLGB@?$DMinit?$DO@ 00000001800054c4     libgetfldmdf004.obj
 0002:000014d0       ??_C@_0BG@IKDDPPGD@?$CILjava?1lang?1String?$DL?$CJV@ 00000001800054d0     libgetfldmdf004.obj
 0002:000014f0       ??_C@_0EB@IFJBFEKC@?$CIthreadClass?5?$DN?5jni_env?9?$DOFindCla@ 00000001800054f0     libgetfldmdf004.obj
 0002:00001540       ??_C@_0GF@FGFIBKKL@?$CIthreadCtor?5?$DN?5jni_env?9?$DOGetMetho@ 0000000180005540     libgetfldmdf004.obj
 0002:000015a8       ??_C@_0DN@NCPDJLOG@?$CIthreadName?5?$DN?5jni_env?9?$DONewStrin@ 00000001800055a8     libgetfldmdf004.obj
 0002:000015f0       ??_C@_0FE@PFKODBGC@?$CIthreadObject?5?$DN?5jni_env?9?$DONewObj@ 00000001800055f0     libgetfldmdf004.obj
 0002:00001650       ??_C@_0ED@HOBAHHJI@?$CIthreadGlobalRef?5?$DN?5jni_env?9?$DONew@ 0000000180005650     libgetfldmdf004.obj
 0002:000016a0       ??_C@_0FN@HNJJAHFC@jvmti_env?9?$DORunAgentThread?$CIagent@ 00000001800056a0     libgetfldmdf004.obj
 0002:00001700       ??_C@_0EA@MOJDNKDF@Debuggee?5status?5sync?5aborted?5be@ 0000000180005700     libgetfldmdf004.obj
 0002:00001740       ??_C@_0EA@EEOEJAEN@status?5?$DN?5syncDebuggeeStatus?$CIjni@ 0000000180005740     libgetfldmdf004.obj
 0002:00001780       ??_C@_0BL@JBCFNBMB@nsk_jvmti_resetAgentData?$CI?$CJ@ 0000000180005780     libgetfldmdf004.obj
 0002:000017a0       ??_C@_0EL@LPBEELIP@s?2test?2hotspot?2jtreg?2vmTestbase@ 00000001800057a0     libgetfldmdf004.obj
 0002:000017f0       ??_C@_0CK@JDAMFDMJ@jvmti?9?$DOSetTag?$CIo?0?5tag?$CJ?5?$DN?$DN?5JVMTI_@ 00000001800057f0     libgetfldmdf004.obj
 0002:00001820       ??_C@_0CC@DAMNHKNI@Can?8t?5set?5tag?5?$CFli?5for?5object?5?$CFl@ 0000000180005820     libgetfldmdf004.obj
 0002:00001848       ??_C@_0DL@HAJPNKEF@jvmti?9?$DOGetObjectHashCode?$CIo?0?5?$CGha@ 0000000180005848     libgetfldmdf004.obj
 0002:00001888       ??_C@_0BL@JFPIEOBF@Can?8t?5get?5hash?5object?5?$CFlx?6@ 0000000180005888     libgetfldmdf004.obj
 0002:000018a8       ??_C@_0BG@DICPHBKN@setTag?3?5?$CF08x?5?$DM?9?5?$CF?53li@ 00000001800058a8     libgetfldmdf004.obj
 0002:000018c0       ??_C@_0DH@FCEEBDMJ@?$CIs?5?$DN?5jni?9?$DOGetStringUTFChars?$CIsIn@ 00000001800058c0     libgetfldmdf004.obj
 0002:000018f8       ??_C@_0BJ@OKKGHDCN@Can?8t?5get?5string?5at?5?$CF?$CDp?6@ 00000001800058f8     libgetfldmdf004.obj
 0002:00001918       ??_C@_0BP@EKFLGGFJ@Can?8t?5get?5string?5at?5?$CF?$CDp?3?5null?6@ 0000000180005918     libgetfldmdf004.obj
 0002:00001938       ??_C@_06ICODBHCL@?5?1?1?5?$CFs@ 0000000180005938     libgetfldmdf004.obj
 0002:00001940       ??_C@_0DB@KGFPLEGO@?$CIr?5?$DN?5jvmti?9?$DOGetTag?$CIo?0?5?$CGtag?$CJ?$CJ?5?$DN?$DN@ 0000000180005940     libgetfldmdf004.obj
 0002:00001978       ??_C@_0CO@PDAGBCGJ@Can?8t?5GetTag?5for?5object?5?$CFlx?4?5Re@ 0000000180005978     libgetfldmdf004.obj
 0002:000019a8       ??_C@_0CH@HPEODOHC@TEST_BUG?3?5Max?4?5number?5of?5refs?5r@ 00000001800059a8     libgetfldmdf004.obj
 0002:000019d0       ??_C@_0DI@PHFCABIM@?$CIr?5?$DN?5jvmti?9?$DOGetTag?$CIfrom?0?5?$CGtagFr@ 00000001800059d0     libgetfldmdf004.obj
 0002:00001a08       ??_C@_0DI@MDEGFNKD@TEST_BUG?3?5Can?8t?5GetTag?5for?5obje@ 0000000180005a08     libgetfldmdf004.obj
 0002:00001a40       ??_C@_0DE@MLELJAHM@?$CIr?5?$DN?5jvmti?9?$DOGetTag?$CIto?0?5?$CGtagTo?$CJ?$CJ@ 0000000180005a40     libgetfldmdf004.obj
 0002:00001a78       ??_C@_09OPJEJKBL@printdump@ 0000000180005a78     libgetfldmdf004.obj
 0002:00001a88       ??_C@_0CJ@KCDEKOCJ@Wrong?5result?5of?5a?5valid?5call?5to@ 0000000180005a88     libgetfldmdf004.obj
 0002:00001ab8       ??_C@_07ELNDHEBG@?5PUBLIC@ 0000000180005ab8     libgetfldmdf004.obj
 0002:00001ac0       ??_C@_08CAHMABBB@?5PRIVATE@ 0000000180005ac0     libgetfldmdf004.obj
 0002:00001ad0       ??_C@_0L@DGJONHAA@?5PROTECTED@ 0000000180005ad0     libgetfldmdf004.obj
 0002:00001ae0       ??_C@_07GDGKLIIO@?5STATIC@ 0000000180005ae0     libgetfldmdf004.obj
 0002:00001ae8       ??_C@_06HHJDACKE@?5FINAL@  0000000180005ae8     libgetfldmdf004.obj
 0002:00001af0       ??_C@_06OCBGFMKA@?5SUPER@  0000000180005af0     libgetfldmdf004.obj
 0002:00001af8       ??_C@_09DKHDALHI@?5VOLATILE@ 0000000180005af8     libgetfldmdf004.obj
 0002:00001b08       ??_C@_0L@NIFMJCKF@?5TRANSIENT@ 0000000180005b08     libgetfldmdf004.obj
 0002:00001b18       ??_C@_07HNCLACND@?5NATIVE@ 0000000180005b18     libgetfldmdf004.obj
 0002:00001b20       ??_C@_0L@OLMLCBEN@?5INTERFACE@ 0000000180005b20     libgetfldmdf004.obj
 0002:00001b30       ??_C@_09LJCLPHHM@?5ABSTRACT@ 0000000180005b30     libgetfldmdf004.obj
 0002:00001b40       ??_C@_09KFPDEIEG@?5?$CI0x?$CF0x?$CJ?6@ 0000000180005b40     libgetfldmdf004.obj
 0002:00001b50       ??_C@_0CH@CDOJMNAO@JVMTI?5client?5was?5not?5properly?5l@ 0000000180005b50     libgetfldmdf004.obj
 0002:00001b78       ??_C@_0CG@BCDHGIMH@?$CI?$CFd?$CJ?5cannot?5get?5field?5ID?5for?5?$CFs@ 0000000180005b78     libgetfldmdf004.obj
 0002:00001ba0       ??_C@_0DC@HIGNKPIG@?$CIGetFieldModifiers?$CD?$CFd?$CJ?5unexpect@ 0000000180005ba0     libgetfldmdf004.obj
 0002:00001bd8       ??_C@_08KJMGEHLM@?$DO?$DO?$DO?5?$CF2d?3@ 0000000180005bd8     libgetfldmdf004.obj
 0002:00001be8       ??_C@_0BN@DOGCLOOC@?$CI?$CF2d?$CJ?5access?5flags?5expected?3@ 0000000180005be8     libgetfldmdf004.obj
 0002:00001c08       ??_C@_0O@LEOGAMKC@?7?7?5?5?5?5actual?3@ 0000000180005c08     libgetfldmdf004.obj
 0002:00001c30       ??_C@_1EC@JIJBPKFM@?$AAa?$AAp?$AAi?$AA?9?$AAm?$AAs?$AA?9?$AAw?$AAi?$AAn?$AA?9?$AAc?$AAo?$AAr?$AAe@ 0000000180005c30     MSVCRT:thread_safe_statics.obj
 0002:00001c78       ??_C@_1BK@MGMFAEKH@?$AAk?$AAe?$AAr?$AAn?$AAe?$AAl?$AA3?$AA2?$AA?4?$AAd?$AAl?$AAl@ 0000000180005c78     MSVCRT:thread_safe_statics.obj
 0002:00001c98       ??_C@_0BJ@JEBJOJFJ@SleepConditionVariableCS@ 0000000180005c98     MSVCRT:thread_safe_statics.obj
 0002:00001cb8       ??_C@_0BJ@PGPPEPCC@WakeAllConditionVariable@ 0000000180005cb8     MSVCRT:thread_safe_statics.obj
 0002:00001cd8       _pDefaultRawDllMain        0000000180005cd8     MSVCRT:dll_dllmain.obj
 0002:00001cd8       _pRawDllMain               0000000180005cd8     MSVCRT:dll_dllmain.obj
 0002:00001ce0       __xmm@ffffffffffffffffffffffffffffffff 0000000180005ce0     MSVCRT:utility.obj
 0002:00001cf0       _load_config_used          0000000180005cf0     MSVCRT:loadcfg.obj
 0002:00001f00       _tls_used                  0000000180005f00     MSVCRT:tlssup.obj
 0002:00001f28       __volatile_metadata        0000000180005f28     <linker-defined>
 0002:000022e8       __rtc_iaa                  00000001800062e8     MSVCRT:initsect.obj
 0002:000022f0       __rtc_izz                  00000001800062f0     MSVCRT:initsect.obj
 0002:000022f8       __rtc_taa                  00000001800062f8     MSVCRT:initsect.obj
 0002:00002300       __rtc_tzz                  0000000180006300     MSVCRT:initsect.obj
 0002:00002308       _tls_start                 0000000180006308     MSVCRT:tlssup.obj
 0002:0000230c       _Init_thread_epoch         000000018000630c     MSVCRT:thread_safe_statics.obj
 0002:00002310       _tls_end                   0000000180006310     MSVCRT:tlssup.obj
 0002:000029e4       __IMPORT_DESCRIPTOR_KERNEL32 00000001800069e4     kernel32:KERNEL32.dll
 0002:000029f8       __IMPORT_DESCRIPTOR_VCRUNTIME140 00000001800069f8     vcruntime:VCRUNTIME140.dll
 0002:00002a0c       __IMPORT_DESCRIPTOR_api-ms-win-crt-runtime-l1-1-0 0000000180006a0c     ucrt:api-ms-win-crt-runtime-l1-1-0.dll
 0002:00002a20       __IMPORT_DESCRIPTOR_api-ms-win-crt-stdio-l1-1-0 0000000180006a20     ucrt:api-ms-win-crt-stdio-l1-1-0.dll
 0002:00002a34       __IMPORT_DESCRIPTOR_api-ms-win-crt-string-l1-1-0 0000000180006a34     ucrt:api-ms-win-crt-string-l1-1-0.dll
 0002:00002a48       __NULL_IMPORT_DESCRIPTOR   0000000180006a48     kernel32:KERNEL32.dll
 0003:000004b0       _Init_global_epoch         00000001800084b0     MSVCRT:thread_safe_statics.obj
 0003:000004c0       __security_cookie          00000001800084c0     MSVCRT:gs_cookie.obj
 0003:000004c8       __security_cookie_complement 00000001800084c8     MSVCRT:gs_cookie.obj
 0003:000004d0       __scrt_native_dllmain_reason 00000001800084d0     MSVCRT:utility.obj
 0003:000004d8       __isa_available            00000001800084d8     MSVCRT:cpu_disp.obj
 0003:000004dc       __isa_enabled              00000001800084dc     MSVCRT:cpu_disp.obj
 0003:000004e0       __memset_fast_string_threshold 00000001800084e0     MSVCRT:cpu_disp.obj
 0003:000004e8       __memset_nt_threshold      00000001800084e8     MSVCRT:cpu_disp.obj
 0003:000004f0       __scrt_ucrt_dll_is_in_use  00000001800084f0     MSVCRT:ucrt_stubs.obj
 0003:00000500       g_wrongHeapCallbacks       0000000180008500     libgetfldmdf004.obj
 0003:00000580       g_szTagInfo                0000000180008580     libgetfldmdf004.obj
 0003:000024c0       g_tagFlags                 000000018000a4c0     libgetfldmdf004.obj
 0003:000028a8       g_refsToVerifyCnt          000000018000a8a8     libgetfldmdf004.obj
 0003:000028ac       g_fakeUserData             000000018000a8ac     libgetfldmdf004.obj
 0003:000028b0       g_tagVisitCount            000000018000a8b0     libgetfldmdf004.obj
 0003:00003850       g_refsToVerify             000000018000b850     libgetfldmdf004.obj
 0003:0001af50       g_userDataError            0000000180022f50     libgetfldmdf004.obj
 0003:0001b0f0       ?_OptionsStorage@?1??__local_stdio_printf_options@@9@4_KA 00000001800230f0     libgetfldmdf004.obj
 0003:0001b6b8       _tls_index                 00000001800236b8     MSVCRT:tlssup.obj
 0003:0001b6c0       __scrt_current_native_startup_state 00000001800236c0     MSVCRT:utility.obj
 0003:0001b6c8       __scrt_native_startup_lock 00000001800236c8     MSVCRT:utility.obj
 0003:0001b708       __scrt_debugger_hook_flag  0000000180023708     MSVCRT:utility_desktop.obj
 0003:0001b710       ?__type_info_root_node@@3U__type_info_node@@A 0000000180023710     MSVCRT:tncleanup.obj
 0003:0001b720       ?_OptionsStorage@?1??__local_stdio_scanf_options@@9@4_KA 0000000180023720     MSVCRT:default_local_stdio_options.obj
 0003:0001b728       __favor                    0000000180023728     MSVCRT:cpu_disp.obj
 0003:0001b730       __dyn_tls_init_callback    0000000180023730     <common>

 entry point at        0001:000022f0

 Static symbols

 0000:fffda000       .debug$S                   0000000180000000     getfldmdf004.exp
 0000:fffda000       .debug$S                   0000000180000000     vcruntime:VCRUNTIME140.dll
 0000:fffda000       .debug$S                   0000000180000000     vcruntime:VCRUNTIME140.dll
 0000:fffda000       .debug$S                   0000000180000000     vcruntime:VCRUNTIME140.dll
 0000:fffda000       .debug$S                   0000000180000000     vcruntime:VCRUNTIME140.dll
 0000:fffda000       .debug$S                   0000000180000000     vcruntime:VCRUNTIME140.dll
 0000:fffda000       .debug$S                   0000000180000000     vcruntime:VCRUNTIME140.dll
 0000:fffda000       .debug$S                   0000000180000000     vcruntime:VCRUNTIME140.dll
 0000:fffda000       .debug$S                   0000000180000000     ucrt:api-ms-win-crt-convert-l1-1-0.dll
 0002:ffffc000       .idata$6                   0000000180000000     ucrt:api-ms-win-crt-convert-l1-1-0.dll
 0000:fffda000       .debug$S                   0000000180000000     ucrt:api-ms-win-crt-heap-l1-1-0.dll
 0000:fffda000       .debug$S                   0000000180000000     ucrt:api-ms-win-crt-heap-l1-1-0.dll
 0000:fffda000       .debug$S                   0000000180000000     ucrt:api-ms-win-crt-heap-l1-1-0.dll
 0000:fffda000       .debug$S                   0000000180000000     ucrt:api-ms-win-crt-heap-l1-1-0.dll
 0002:ffffc000       .idata$6                   0000000180000000     ucrt:api-ms-win-crt-heap-l1-1-0.dll
 0000:fffda000       .debug$S                   0000000180000000     ucrt:api-ms-win-crt-runtime-l1-1-0.dll
 0000:fffda000       .debug$S                   0000000180000000     ucrt:api-ms-win-crt-runtime-l1-1-0.dll
 0000:fffda000       .debug$S                   0000000180000000     ucrt:api-ms-win-crt-runtime-l1-1-0.dll
 0000:fffda000       .debug$S                   0000000180000000     ucrt:api-ms-win-crt-runtime-l1-1-0.dll
 0000:fffda000       .debug$S                   0000000180000000     ucrt:api-ms-win-crt-runtime-l1-1-0.dll
 0000:fffda000       .debug$S                   0000000180000000     ucrt:api-ms-win-crt-runtime-l1-1-0.dll
 0000:fffda000       .debug$S                   0000000180000000     ucrt:api-ms-win-crt-runtime-l1-1-0.dll
 0000:fffda000       .debug$S                   0000000180000000     ucrt:api-ms-win-crt-runtime-l1-1-0.dll
 0000:fffda000       .debug$S                   0000000180000000     ucrt:api-ms-win-crt-runtime-l1-1-0.dll
 0000:fffda000       .debug$S                   0000000180000000     ucrt:api-ms-win-crt-runtime-l1-1-0.dll
 0000:fffda000       .debug$S                   0000000180000000     ucrt:api-ms-win-crt-runtime-l1-1-0.dll
 0000:fffda000       .debug$S                   0000000180000000     ucrt:api-ms-win-crt-runtime-l1-1-0.dll
 0000:fffda000       .debug$S                   0000000180000000     ucrt:api-ms-win-crt-runtime-l1-1-0.dll
 0000:fffda000       .debug$S                   0000000180000000     ucrt:api-ms-win-crt-runtime-l1-1-0.dll
 0000:fffda000       .debug$S                   0000000180000000     ucrt:api-ms-win-crt-runtime-l1-1-0.dll
 0000:fffda000       .debug$S                   0000000180000000     ucrt:api-ms-win-crt-runtime-l1-1-0.dll
 0000:fffda000       .debug$S                   0000000180000000     ucrt:api-ms-win-crt-stdio-l1-1-0.dll
 0000:fffda000       .debug$S                   0000000180000000     ucrt:api-ms-win-crt-stdio-l1-1-0.dll
 0000:fffda000       .debug$S                   0000000180000000     ucrt:api-ms-win-crt-stdio-l1-1-0.dll
 0000:fffda000       .debug$S                   0000000180000000     ucrt:api-ms-win-crt-stdio-l1-1-0.dll
 0000:fffda000       .debug$S                   0000000180000000     ucrt:api-ms-win-crt-stdio-l1-1-0.dll
 0000:fffda000       .debug$S                   0000000180000000     ucrt:api-ms-win-crt-stdio-l1-1-0.dll
 0000:fffda000       .debug$S                   0000000180000000     ucrt:api-ms-win-crt-stdio-l1-1-0.dll
 0000:fffda000       .debug$S                   0000000180000000     ucrt:api-ms-win-crt-stdio-l1-1-0.dll
 0000:fffda000       .debug$S                   0000000180000000     ucrt:api-ms-win-crt-stdio-l1-1-0.dll
 0000:fffda000       .debug$S                   0000000180000000     ucrt:api-ms-win-crt-stdio-l1-1-0.dll
 0000:fffda000       .debug$S                   0000000180000000     ucrt:api-ms-win-crt-string-l1-1-0.dll
 0000:fffda000       .debug$S                   0000000180000000     ucrt:api-ms-win-crt-string-l1-1-0.dll
 0000:fffda000       .debug$S                   0000000180000000     ucrt:api-ms-win-crt-string-l1-1-0.dll
 0000:fffda000       .debug$S                   0000000180000000     ucrt:api-ms-win-crt-string-l1-1-0.dll
 0000:fffda000       .debug$S                   0000000180000000     ucrt:api-ms-win-crt-string-l1-1-0.dll
 0000:fffda000       .debug$S                   0000000180000000     ucrt:api-ms-win-crt-string-l1-1-0.dll
 0000:fffda000       .debug$S                   0000000180000000     ucrt:api-ms-win-crt-string-l1-1-0.dll
 0000:fffda000       .debug$S                   0000000180000000     ucrt:api-ms-win-crt-string-l1-1-0.dll
 0000:fffda000       .debug$S                   0000000180000000     kernel32:KERNEL32.dll
 0000:fffda000       .debug$S                   0000000180000000     kernel32:KERNEL32.dll
 0000:fffda000       .debug$S                   0000000180000000     kernel32:KERNEL32.dll
 0000:fffda000       .debug$S                   0000000180000000     kernel32:KERNEL32.dll
 0000:fffda000       .debug$S                   0000000180000000     kernel32:KERNEL32.dll
 0000:fffda000       .debug$S                   0000000180000000     kernel32:KERNEL32.dll
 0000:fffda000       .debug$S                   0000000180000000     kernel32:KERNEL32.dll
 0000:fffda000       .debug$S                   0000000180000000     kernel32:KERNEL32.dll
 0000:fffda000       .debug$S                   0000000180000000     kernel32:KERNEL32.dll
 0000:fffda000       .debug$S                   0000000180000000     kernel32:KERNEL32.dll
 0000:fffda000       .debug$S                   0000000180000000     kernel32:KERNEL32.dll
 0000:fffda000       .debug$S                   0000000180000000     kernel32:KERNEL32.dll
 0000:fffda000       .debug$S                   0000000180000000     kernel32:KERNEL32.dll
 0000:fffda000       .debug$S                   0000000180000000     kernel32:KERNEL32.dll
 0000:fffda000       .debug$S                   0000000180000000     kernel32:KERNEL32.dll
 0000:fffda000       .debug$S                   0000000180000000     kernel32:KERNEL32.dll
 0000:fffda000       .debug$S                   0000000180000000     kernel32:KERNEL32.dll
 0000:fffda000       .debug$S                   0000000180000000     kernel32:KERNEL32.dll
 0000:fffda000       .debug$S                   0000000180000000     kernel32:KERNEL32.dll
 0000:fffda000       .debug$S                   0000000180000000     kernel32:KERNEL32.dll
 0000:fffda000       .debug$S                   0000000180000000     kernel32:KERNEL32.dll
 0000:fffda000       .debug$S                   0000000180000000     kernel32:KERNEL32.dll
 0000:fffda000       .debug$S                   0000000180000000     kernel32:KERNEL32.dll
 0000:fffda000       .debug$S                   0000000180000000     kernel32:KERNEL32.dll
 0000:fffda000       .debug$S                   0000000180000000     kernel32:KERNEL32.dll
 0000:fffda000       .debug$S                   0000000180000000     kernel32:KERNEL32.dll
 0000:fffda000       .debug$S                   0000000180000000     kernel32:KERNEL32.dll
 0000:fffda000       .debug$S                   0000000180000000     kernel32:KERNEL32.dll
 0001:00000e34       addRefToVerify             0000000180001e34 f   libgetfldmdf004.obj
 0001:00000ea0       agentThreadWrapper         0000000180001ea0 f   libgetfldmdf004.obj
 0001:00001090       file_basename              0000000180002090 f   libgetfldmdf004.obj
 0001:000017d4       startAgentThreadWrapper    00000001800027d4 f   libgetfldmdf004.obj
 0001:00001b14       syncDebuggeeStatus         0000000180002b14 f   libgetfldmdf004.obj
 0001:00001db4       capture_previous_context   0000000180002db4 f   MSVCRT:gs_report.obj
 0001:00001e28       ?__scrt_initialize_thread_safe_statics@@YAHXZ 0000000180002e28 f   MSVCRT:thread_safe_statics.obj
 0001:00001ef8       ?__scrt_uninitialize_thread_safe_statics@@YAXXZ 0000000180002ef8 f   MSVCRT:thread_safe_statics.obj
 0001:00001fa0       $$000000                   0000000180002fa0     MSVCRT:amdsecgs.obj
 0001:00001fd0       ?dllmain_crt_dispatch@@YAHQEAUHINSTANCE__@@KQEAX@Z 0000000180002fd0 f   MSVCRT:dll_dllmain.obj
 0001:00002020       ?dllmain_crt_process_attach@@YAHQEAUHINSTANCE__@@QEAX@Z 0000000180003020 f   MSVCRT:dll_dllmain.obj
 0001:00002138       ?dllmain_crt_process_detach@@YAH_N@Z 0000000180003138 f   MSVCRT:dll_dllmain.obj
 0001:000021bc       ?dllmain_dispatch@@YAHQEAUHINSTANCE__@@KQEAX@Z 00000001800031bc f   MSVCRT:dll_dllmain.obj
 0001:00002bd0       $$000000                   0000000180003bd0     MSVCRT:guard_dispatch.obj
 0001:00002bf0       $$000000                   0000000180003bf0     MSVCRT:guard_xfg_dispatch.obj
 0001:00002c06       ?fin$0@?0??dllmain_crt_process_attach@@YAHQEAUHINSTANCE__@@QEAX@Z@4HA 0000000180003c06 f   MSVCRT:dll_dllmain.obj
 0001:00002c1d       ?fin$0@?0??dllmain_crt_process_detach@@YAH_N@Z@4HA 0000000180003c1d f   MSVCRT:dll_dllmain.obj
 0001:00002c36       ?fin$1@?0??dllmain_crt_process_detach@@YAH_N@Z@4HA 0000000180003c36 f   MSVCRT:dll_dllmain.obj
 0001:00002c4a       ?filt$0@?0??dllmain_dispatch@@YAHQEAUHINSTANCE__@@KQEAX@Z@4HA 0000000180003c4a f   MSVCRT:dll_dllmain.obj
 0001:00002c80       __scrt_is_nonwritable_in_current_image$filt$0 0000000180003c80 f   MSVCRT:utility.obj
 0002:000001e8       ?__scrt_initialize_tss_var@@3P6AHXZEA 00000001800041e8     MSVCRT:thread_safe_statics.obj
 0002:00000310       ?opcLengths@@3QBEB         0000000180004310     libgetfldmdf004.obj
 0002:00001c18       GS_ExceptionPointers       0000000180005c18     MSVCRT:gs_report.obj
 0002:00002318       $unwind$fprintf            0000000180006318     libgetfldmdf004.obj
 0002:00002324       $unwind$printf             0000000180006324     libgetfldmdf004.obj
 0002:00002330       $unwind$?NewObject@JNIEnv_@@QEAAPEAV_jobject@@PEAV_jclass@@PEAU_jmethodID@@ZZ 0000000180006330     libgetfldmdf004.obj
 0002:00002330       $unwind$nsk_lcomplain      0000000180006330     libgetfldmdf004.obj
 0002:00002330       $unwind$nsk_ldisplay       0000000180006330     libgetfldmdf004.obj
 0002:00002338       $unwind$nsk_lvdisplay      0000000180006338     libgetfldmdf004.obj
 0002:00002338       $unwind$_RTC_Initialize    0000000180006338     MSVCRT:initsect.obj
 0002:00002338       $unwind$_RTC_Terminate     0000000180006338     MSVCRT:initsect.obj
 0002:00002338       $unwind$?__scrt_initialize_thread_safe_statics@@YAHXZ 0000000180006338     MSVCRT:thread_safe_statics.obj
 0002:00002344       $unwind$nsk_lvcomplain     0000000180006344     libgetfldmdf004.obj
 0002:0000235c       $unwind$nsk_ltrace         000000018000635c     libgetfldmdf004.obj
 0002:0000235c       $unwind$__report_gsfailure 000000018000635c     MSVCRT:gs_report.obj
 0002:00002364       $unwind$Agent_Initialize   0000000180006364     libgetfldmdf004.obj
 0002:00002364       $unwind$nsk_lvtrace        0000000180006364     libgetfldmdf004.obj
 0002:00002364       $unwind$printModifiers     0000000180006364     libgetfldmdf004.obj
 0002:00002364       $unwind$__raise_securityfailure 0000000180006364     MSVCRT:gs_report.obj
 0002:00002364       $unwind$__scrt_initialize_crt 0000000180006364     MSVCRT:utility.obj
 0002:00002364       $unwind$__scrt_initialize_onexit_tables 0000000180006364     MSVCRT:utility.obj
 0002:00002364       $unwind$__scrt_release_startup_lock 0000000180006364     MSVCRT:utility.obj
 0002:00002364       $unwind$__scrt_uninitialize_crt 0000000180006364     MSVCRT:utility.obj
 0002:00002364       $unwind$_onexit            0000000180006364     MSVCRT:utility.obj
 0002:0000236c       $unwind$nsk_lverify        000000018000636c     libgetfldmdf004.obj
 0002:0000237c       $unwind$nsk_vprintf        000000018000637c     libgetfldmdf004.obj
 0002:0000238c       $unwind$nsk_printf         000000018000638c     libgetfldmdf004.obj
 0002:00002394       $unwind$?nsk_jni_lverify@@YAHHPEAUJNIEnv_@@HQEBDH1ZZ 0000000180006394     libgetfldmdf004.obj
 0002:000023a8       $unwind$?nsk_jni_check_exception@@YAHPEAUJNIEnv_@@QEBDH@Z 00000001800063a8     libgetfldmdf004.obj
 0002:000023c4       $unwind$Java_nsk_jvmti_unit_FollowReferences_FollowRefObjects_resetTags 00000001800063c4     libgetfldmdf004.obj
 0002:000023c4       $unwind$addRefToVerify     00000001800063c4     libgetfldmdf004.obj
 0002:000023c4       $unwind$nsk_jvmti_resetAgentData 00000001800063c4     libgetfldmdf004.obj
 0002:000023c4       $unwind$nsk_jvmti_setFailStatus 00000001800063c4     libgetfldmdf004.obj
 0002:000023c4       $unwind$__scrt_initialize_default_local_stdio_options 00000001800063c4     MSVCRT:default_local_stdio_options.obj
 0002:000023c4       $unwind$?dllmain_crt_dispatch@@YAHQEAUHINSTANCE__@@KQEAX@Z 00000001800063c4     MSVCRT:dll_dllmain.obj
 0002:000023c4       $unwind$DllMain            00000001800063c4     MSVCRT:dll_dllmain_stub.obj
 0002:000023c4       $unwind$__GSHandlerCheck   00000001800063c4     MSVCRT:gshandler.obj
 0002:000023c4       $unwind$?__scrt_uninitialize_thread_safe_statics@@YAXXZ 00000001800063c4     MSVCRT:thread_safe_statics.obj
 0002:000023c4       $unwind$__scrt_acquire_startup_lock 00000001800063c4     MSVCRT:utility.obj
 0002:000023c4       $unwind$__scrt_dllmain_after_initialize_c 00000001800063c4     MSVCRT:utility.obj
 0002:000023c4       $unwind$__scrt_dllmain_before_initialize_c 00000001800063c4     MSVCRT:utility.obj
 0002:000023c4       $unwind$__scrt_dllmain_crt_thread_attach 00000001800063c4     MSVCRT:utility.obj
 0002:000023c4       $unwind$__scrt_dllmain_crt_thread_detach 00000001800063c4     MSVCRT:utility.obj
 0002:000023c4       $unwind$__scrt_dllmain_uninitialize_c 00000001800063c4     MSVCRT:utility.obj
 0002:000023c4       $unwind$__scrt_dllmain_uninitialize_critical 00000001800063c4     MSVCRT:utility.obj
 0002:000023c4       $unwind$atexit             00000001800063c4     MSVCRT:utility.obj
 0002:000023cc       $unwind$nsk_jvmti_lverify  00000001800063cc     libgetfldmdf004.obj
 0002:000023e0       $unwind$exitOnError        00000001800063e0     libgetfldmdf004.obj
 0002:000023f0       $unwind$Java_nsk_share_jvmti_ArgumentHandler_getAgentOptionsString 00000001800063f0     libgetfldmdf004.obj
 0002:00002404       $unwind$Java_nsk_jvmti_unit_FollowReferences_FollowRefObjects_getTag 0000000180006404     libgetfldmdf004.obj
 0002:00002404       $unwind$Java_nsk_share_jvmti_DebugeeClass_checkStatus 0000000180006404     libgetfldmdf004.obj
 0002:00002404       $unwind$agentThreadWrapper 0000000180006404     libgetfldmdf004.obj
 0002:00002414       $unwind$startAgentThreadWrapper 0000000180006414     libgetfldmdf004.obj
 0002:00002430       $unwind$syncDebuggeeStatus 0000000180006430     libgetfldmdf004.obj
 0002:00002430       $unwind$__scrt_dllmain_exception_filter 0000000180006430     MSVCRT:utility.obj
 0002:00002444       $unwind$Java_nsk_share_jvmti_DebugeeClass_resetAgentData 0000000180006444     libgetfldmdf004.obj
 0002:0000244c       $unwind$MA_checkStatus     000000018000644c     libgetfldmdf004.obj
 0002:00002460       $unwind$Java_nsk_jvmti_unit_FollowReferences_FollowRefObjects_setTag 0000000180006460     libgetfldmdf004.obj
 0002:00002478       $unwind$Java_nsk_jvmti_unit_FollowReferences_FollowRefObjects_addRefToVerify 0000000180006478     libgetfldmdf004.obj
 0002:00002494       $unwind$Java_nsk_jvmti_GetFieldModifiers_getfldmdf004_check 0000000180006494     libgetfldmdf004.obj
 0002:000024ac       $unwind$capture_previous_context 00000001800064ac     MSVCRT:gs_report.obj
 0002:000024b8       $unwind$__GSHandlerCheckCommon 00000001800064b8     MSVCRT:gshandler.obj
 0002:000024c0       $xdatasym                  00000001800064c0     MSVCRT:amdsecgs.obj
 0002:000024c4       $unwind$?dllmain_crt_process_attach@@YAHQEAUHINSTANCE__@@QEAX@Z 00000001800064c4     MSVCRT:dll_dllmain.obj
 0002:00002500       $unwind$?fin$0@?0??dllmain_crt_process_attach@@YAHQEAUHINSTANCE__@@QEAX@Z@4HA 0000000180006500     MSVCRT:dll_dllmain.obj
 0002:00002500       $unwind$?fin$0@?0??dllmain_crt_process_detach@@YAH_N@Z@4HA 0000000180006500     MSVCRT:dll_dllmain.obj
 0002:00002500       $unwind$?fin$1@?0??dllmain_crt_process_detach@@YAH_N@Z@4HA 0000000180006500     MSVCRT:dll_dllmain.obj
 0002:00002508       $unwind$?dllmain_crt_process_detach@@YAH_N@Z 0000000180006508     MSVCRT:dll_dllmain.obj
 0002:0000255c       $unwind$?dllmain_dispatch@@YAHQEAUHINSTANCE__@@KQEAX@Z 000000018000655c     MSVCRT:dll_dllmain.obj
 0002:00002584       $unwind$?filt$0@?0??dllmain_dispatch@@YAHQEAUHINSTANCE__@@KQEAX@Z@4HA 0000000180006584     MSVCRT:dll_dllmain.obj
 0002:0000258c       $unwind$_DllMainCRTStartup 000000018000658c     MSVCRT:dll_dllmain.obj
 0002:0000259c       $unwind$__scrt_is_nonwritable_in_current_image 000000018000659c     MSVCRT:utility.obj
 0002:000025bc       $unwind$__scrt_is_nonwritable_in_current_image$filt$0 00000001800065bc     MSVCRT:utility.obj
 0002:000025c4       $unwind$__scrt_fastfail    00000001800065c4     MSVCRT:utility_desktop.obj
 0002:000025d4       $unwind$__security_init_cookie 00000001800065d4     MSVCRT:gs_support.obj
 0002:000025e0       $unwind$__isa_available_init 00000001800065e0     MSVCRT:cpu_disp.obj
 0002:000025f0       $xdatasym                  00000001800065f0     MSVCRT:guard_dispatch.obj
 0002:000025f8       $xdatasym                  00000001800065f8     MSVCRT:guard_xfg_dispatch.obj
 0002:00002600       .edata                     0000000180006600     getfldmdf004.exp
 0002:00002628       rgpv                       0000000180006628     getfldmdf004.exp
 0002:00002668       rgszName                   0000000180006668     getfldmdf004.exp
 0002:000026a8       rgwOrd                     00000001800066a8     getfldmdf004.exp
 0002:000026c8       szName                     00000001800066c8     getfldmdf004.exp
 0002:000026d9       $N00001                    00000001800066d9     getfldmdf004.exp
 0002:000026e8       $N00002                    00000001800066e8     getfldmdf004.exp
 0002:000026f5       $N00003                    00000001800066f5     getfldmdf004.exp
 0002:00002729       $N00004                    0000000180006729     getfldmdf004.exp
 0002:0000275e       $N00005                    000000018000675e     getfldmdf004.exp
 0002:000027a3       $N00006                    00000001800067a3     getfldmdf004.exp
 0002:000027e0       $N00007                    00000001800067e0     getfldmdf004.exp
 0002:00002828       $N00008                    0000000180006828     getfldmdf004.exp
 0002:00002868       $N00009                    0000000180006868     getfldmdf004.exp
 0002:000028a5       $N00010                    00000001800068a5     getfldmdf004.exp
 0002:000028e0       $N00011                    00000001800068e0     getfldmdf004.exp
 0002:0000290e       $N00012                    000000018000690e     getfldmdf004.exp
 0002:0000293f       $N00013                    000000018000693f     getfldmdf004.exp
 0002:0000296e       $N00014                    000000018000696e     getfldmdf004.exp
 0002:0000299d       $N00015                    000000018000699d     getfldmdf004.exp
 0002:000029d2       $N00016                    00000001800069d2     getfldmdf004.exp
 0002:00002de2       .idata$6                   0000000180006de2     kernel32:KERNEL32.dll
 0002:00002e46       .idata$6                   0000000180006e46     vcruntime:VCRUNTIME140.dll
 0002:00002fb2       .idata$6                   0000000180006fb2     ucrt:api-ms-win-crt-runtime-l1-1-0.dll
 0002:00002fd4       .idata$6                   0000000180006fd4     ucrt:api-ms-win-crt-stdio-l1-1-0.dll
 0002:00002ff4       .idata$6                   0000000180006ff4     ucrt:api-ms-win-crt-string-l1-1-0.dll
 0003:00000000       ?codeAttributeName@@3PEBDEB 0000000180008000     libgetfldmdf004.obj
 0003:00000008       ?lineNumberAttributeName@@3PEBDEB 0000000180008008     libgetfldmdf004.obj
 0003:00000010       ?localVarAttributeName@@3PEBDEB 0000000180008010     libgetfldmdf004.obj
 0003:00000018       ?localVarTypeAttributeName@@3PEBDEB 0000000180008018     libgetfldmdf004.obj
 0003:00000020       ?stackMapAttributeName@@3PEBDEB 0000000180008020     libgetfldmdf004.obj
 0003:00000028       ?callBytes@@3PAEA          0000000180008028     libgetfldmdf004.obj
 0003:0000002c       ?allocBytes@@3PAEA         000000018000802c     libgetfldmdf004.obj
 0003:00000030       fields                     0000000180008030     libgetfldmdf004.obj
 0003:0001af54       redefineAttempted          0000000180022f54     libgetfldmdf004.obj
 0003:0001af58       nsk_context                0000000180022f58     libgetfldmdf004.obj
 0003:0001af64       redefineSucceed            0000000180022f64     libgetfldmdf004.obj
 0003:0001af68       agentFailed                0000000180022f68     libgetfldmdf004.obj
 0003:0001af6c       currentAgentStatus         0000000180022f6c     libgetfldmdf004.obj
 0003:0001af70       context                    0000000180022f70     libgetfldmdf004.obj
 0003:0001b028       agentThread                0000000180023028     libgetfldmdf004.obj
 0003:0001b030       agentThreadProc            0000000180023030     libgetfldmdf004.obj
 0003:0001b038       agentThreadArg             0000000180023038     libgetfldmdf004.obj
 0003:0001b040       agent_data                 0000000180023040     libgetfldmdf004.obj
 0003:0001b050       jvmti_env                  0000000180023050     libgetfldmdf004.obj
 0003:0001b058       jvm                        0000000180023058     libgetfldmdf004.obj
 0003:0001b060       jni_env                    0000000180023060     libgetfldmdf004.obj
 0003:0001b068       checkStatus_func           0000000180023068     libgetfldmdf004.obj
 0003:0001b070       ?codeAttributeIndex@@3GA   0000000180023070     libgetfldmdf004.obj
 0003:0001b072       printdump                  0000000180023072     libgetfldmdf004.obj
 0003:0001b074       ?lineNumberAttributeIndex@@3GA 0000000180023074     libgetfldmdf004.obj
 0003:0001b078       ?localVarAttributeIndex@@3GA 0000000180023078     libgetfldmdf004.obj
 0003:0001b07c       ?localVarTypeAttributeIndex@@3GA 000000018002307c     libgetfldmdf004.obj
 0003:0001b080       ?stackMapAttributeIndex@@3GA 0000000180023080     libgetfldmdf004.obj
 0003:0001b084       ?stackFrameOffset@@3GA     0000000180023084     libgetfldmdf004.obj
 0003:0001b088       ?mode@@3HA                 0000000180023088     libgetfldmdf004.obj
 0003:0001b08c       ?constantPoolSize@@3GA     000000018002308c     libgetfldmdf004.obj
 0003:0001b090       ?orig@@3PEBEEB             0000000180023090     libgetfldmdf004.obj
 0003:0001b098       ?gen@@3PEAEEA              0000000180023098     libgetfldmdf004.obj
 0003:0001b0a0       ?inputPos@@3PEAEEA         00000001800230a0     libgetfldmdf004.obj
 0003:0001b0a8       ?endPos@@3PEBEEB           00000001800230a8     libgetfldmdf004.obj
 0003:0001b0b0       ?genPos@@3PEAEEA           00000001800230b0     libgetfldmdf004.obj
 0003:0001b0b8       ?markPos@@3PEAEEA          00000001800230b8     libgetfldmdf004.obj
 0003:0001b0c0       ?constantPool@@3PEAPEADEA  00000001800230c0     libgetfldmdf004.obj
 0003:0001b0c8       ?constantPoolCount@@3GA    00000001800230c8     libgetfldmdf004.obj
 0003:0001b0cc       ?zeroBytes@@3PAEA          00000001800230cc     libgetfldmdf004.obj
 0003:0001b0d0       ?codeLength@@3IA           00000001800230d0     libgetfldmdf004.obj
 0003:0001b0d4       result                     00000001800230d4     libgetfldmdf004.obj
 0003:0001b0d8       ?map@@3PEAIEA              00000001800230d8     libgetfldmdf004.obj
 0003:0001b0e0       ?widening@@3PEACEA         00000001800230e0     libgetfldmdf004.obj
 0003:0001b0e8       jvmti                      00000001800230e8     libgetfldmdf004.obj
 0003:0001b100       GS_ExceptionRecord         0000000180023100     MSVCRT:gs_report.obj
 0003:0001b1a0       GS_ContextRecord           00000001800231a0     MSVCRT:gs_report.obj
 0003:0001b670       ?g_tss_cv@@3U_RTL_CONDITION_VARIABLE@@A 0000000180023670     MSVCRT:thread_safe_statics.obj
 0003:0001b678       ?g_tss_event@@3PEAXEA      0000000180023678     MSVCRT:thread_safe_statics.obj
 0003:0001b680       ?g_tss_mutex@@3U_RTL_CRITICAL_SECTION@@A 0000000180023680     MSVCRT:thread_safe_statics.obj
 0003:0001b6a8       ?g_sleep_condition_variable_cs@@3P6AHPEAU_RTL_CONDITION_VARIABLE@@PEAU_RTL_CRITICAL_SECTION@@K@ZEA 00000001800236a8     MSVCRT:thread_safe_statics.obj
 0003:0001b6b0       ?g_wake_all_condition_variable@@3P6AXPEAU_RTL_CONDITION_VARIABLE@@@ZEA 00000001800236b0     MSVCRT:thread_safe_statics.obj
 0003:0001b6bc       ?__proc_attached@@3HA      00000001800236bc     MSVCRT:dll_dllmain.obj
 0003:0001b6d0       ?is_initialized_as_dll@@3_NA 00000001800236d0     MSVCRT:utility.obj
 0003:0001b6d1       ?module_local_atexit_table_initialized@@3_NA 00000001800236d1     MSVCRT:utility.obj
 0003:0001b6d8       ?module_local_atexit_table@@3U_onexit_table_t@@A 00000001800236d8     MSVCRT:utility.obj
 0003:0001b6f0       ?module_local_at_quick_exit_table@@3U_onexit_table_t@@A 00000001800236f0     MSVCRT:utility.obj
